:1000000017EF01F0FFFFFFFF04C03AF003C039F023
:1000100002C038F001C037F000C036F0E9CF30F050
:10002000EACF31F0E1CF32F0E2CF33F0F2A202D0EA
:10003000D1EC00F030C0E9FF31C0EAFF32C0E1FF8F
:1000400033C0E2FF3AC004F039C003F038C002F018
:1000500037C001F036C000F0110097D081A202D065
:10006000800E162617C002F017060250000A03E0A1
:100070001632169E04D0010E156E050E176E90D026
:1000800081A202D0800E182617C002F01706025077
:10009000000A03E01832189E08D0020E156E1832BE
:1000A000189E1832189E070E176E7AD081A202D0C1
:1000B000800E192617C002F017060250000A03E04E
:1000C0001932199E61D0156A070E176E1650700A04
:1000D00058E1800E1914026E0250800A2BE1010EC5
:1000E000046E18C000F0000E016E045005E00036EA
:1000F00000900136FF0FFAD71A0E0024046E000E8E
:100100000120056E7F0E1914026E04C0E9FF05C0C0
:10011000EAFFEECF00F0EECF01F00250005E000EDD
:10012000015A04C0E1FF05C0E2FF00C0E6FF01C0C4
:10013000E6FF27D0010E046E18C000F0000E016E1D
:10014000045005E0003600900136FF0FFAD71A0E72
:100150000024026E000E0120036E02C0E9FF03C0FE
:10016000EAFFEECF00F0EECF01F019500026D8B034
:10017000012A02C0E1FF03C0E2FF00C0E6FF01C0A8
:10018000E6FF166A186A196A0BD01550000AD8B42F
:1001900065D71550010AD8B473D71550020A86E006
:1001A00012002DEC00F0F292F2881200F18CF29223
:1001B000F288156A166A186A196A070E176E120015
:1001C000806A816A826A926A030E936E946A070E4D
:1001D000C16ED6EC00F01A6A1B6A1C6A1D6A1E6AA0
:1001E0001F6A206A216AD09EF28EF28C1200800E65
:1001F000006E800E3518005C02E13450000805E204
:10020000010E345E000E355AF2D71200010E226E36
:10021000030E236E020E246E060E256E040E266E4D
:100220000C0E276E080E286E090E296E120006ECC1
:1002300001F0E0EC00F02A6A2B6A000E2B5C02E170
:10024000040E2A5CD8B078D2010E046E2AC000F0E9
:100250002BC001F0045005E0003600900136FF0F7E
:10026000FAD71A0E0024E96E000E0120EA6EEECFD6
:1002700000F0EECF01F0FF0E0014026E01507F0B74
:10028000036E000E006E0350005C02E10250000895
:10029000D8B04FD2010E046E2AC000F02BC001F07E
:1002A000045005E0003600900136FF0FFAD71A0E11
:1002B0000024E96E000E0120EA6EEECF00F0EECFD2
:1002C00001F0000E0014026E0150800B036E03500B
:1002D000800A02E1000E0218D8A492D0010E046E2A
:1002E0002AC000F02BC001F0045005E00036009059
:1002F0000136FF0FFAD71A0E0024E96E000E012016
:10030000EA6EEECF02F0EECF03F0FF0E035C02E1E7
:10031000FD0E025C3CE2010E046E2AC000F02BC010
:1003200001F0045005E0003600900136FF0FFAD7C7
:100330001A0E0024026E000E0120036E02C0E9FFB7
:1003400003C0EAFFEECF00F0EECF01F0020E002670
:10035000000E012202C0E1FF03C0E2FF00C0E6FF81
:1003600001C0E6FF2C0E2A24026E000E2B20036E25
:1003700002C0E9FF03C0EAFFEECF00F0020E005E0C
:1003800002C0E1FF03C0E2FF00C0E6FF38D0010E6B
:10039000046E2AC000F02BC001F0045005E00036C6
:1003A00000900136FF0FFAD71A0E0024026E000EDD
:1003B0000120036E02C0E9FF03C0EAFFEECF00F0A8
:1003C000EECF01F0004A012A02C0E1FF03C0E2FFC4
:1003D00000C0E6FF01C0E6FF2C0E2A24026E000ECC
:1003E0002B20036E02C0E9FF03C0EAFFEECF00F04E
:1003F000000602C0E1FF03C0E2FF00C0E6FF95D0A7
:10040000010E046E2AC000F02BC001F0045005E07C
:10041000003600900136FF0FFAD71A0E0024E96E5D
:10042000000E0120EA6EEECF02F0EECF03F0000ED8
:10043000006E0350005C02E1025003083CE2010E32
:10044000046E2AC000F02BC001F0045005E0003615
:1004500000900136FF0FFAD71A0E0024026E000E2C
:100460000120036E02C0E9FF03C0EAFFEECF00F0F7
:10047000EECF01F0020E005E000E015A02C0E1FF55
:1004800003C0E2FF00C0E6FF01C0E6FF2C0E2A24F5
:10049000026E000E2B20036E02C0E9FF03C0EAFFCC
:1004A000EECF00F0020E002602C0E1FF03C0E2FF23
:1004B00000C0E6FF3AD0010E046E2AC000F02BC047
:1004C00001F0045005E0003600900136FF0FFAD726
:1004D0001A0E0024026E000E0120036E02C0E9FF16
:1004E00003C0EAFFEECF00F0EECF01F0010E005E98
:1004F000000E015A02C0E1FF03C0E2FF00C0E6FFA8
:1005000001C0E6FF2C0E2A24026E000E2B20036E83
:1005100002C0E9FF03C0EAFFEECF00F0002A02C0EC
:10052000E1FF03C0E2FF00C0E6FFE8D08094070EC1
:100530002C14006E220EE96E000EEA6E0050E926C1
:10054000D8B0EA2AEECF04F0010E0414006E000EBB
:1005500000B0020E8018020B801A04C000F0026A7C
:1005600000B2022A000E02B0010E8018010B801AA0
:1005700004C000F0026A00B4022A000E02B0100E9D
:100580008018100B801A04C000F0026A00B6022A1C
:10059000000E02B0080E8018080B801A8084C9D0A3
:1005A0008292070E2D14006E220EE96E000EEA6E86
:1005B0000050E926D8B0EA2AEECF04F0010E041468
:1005C000006E000E00B0010E8218010B821A04C0EA
:1005D00000F0026A00B2022A000E02B0200E80185B
:1005E000200B801A04C000F0026A00B4022A000E38
:1005F00002B0080E8218080B821A04C000F0026ACA
:1006000000B6022A000E02B0040E8218040B821AF1
:1006100082828FD0829C070E2E14006E220EE96E0D
:10062000000EEA6E0050E926D8B0EA2AEECF04F0B8
:10063000010E0414006E000E00B0200E8218200B74
:10064000821A04C000F0026A00B2022A000E02B050
:10065000100E8218100B821A04C000F0026A00B457
:10066000022A000E02B0040E8118040B811A04C085
:1006700000F0026A00B6022A000E02B0800E821854
:10068000800B821A828C55D0819A070E2F14006E2F
:10069000220EE96E000EEA6E0050E926D8B0EA2A72
:1006A000EECF04F0010E0414006E000E00B0100E28
:1006B0008118100B811A04C000F0026A00B2022AED
:1006C000000E02B0080E8118080B811A04C000F059
:1006D000026A00B4022A000E02B0400E8118400BDC
:1006E000811A04C000F0026A00B6022A000E02B0AD
:1006F000800E8118800B811A818A1BD0000E2B1866
:1007000002E1000E2A18D8B411D7000E2B1802E10E
:10071000010E2A18D8B444D7000E2B1802E1020E9D
:100720002A18D8B477D7000E2B1802E1030E2A1826
:10073000ABE02A4A2B2A81D5880E346E130E356E13
:10074000F7EC00F078D5FFD7FFFFFFFFFFFFFFFFBB
:020000040030CA
:0E000000FFFEFEFAFFFEFBFFFFFFFFFFFFFF0C
:00000001FF
